:020000040000FA
:100000001E284E00690078004929820720341D34DB
:1000100020341F3420341F34203420341F34203443
:100020001F34203420341E3420341F3420341F3435
:10003000203420341F3420341F34203483168501AB
:10004000FB30860081138111011581140114811286
:1000500083120F3085008601003081000A303D2177
:100060008C018D018E014B30B0000030B100B20127
:10007000861C47285B209E018E158B178B167520DA
:1000800003194428061842287C20CF203F286820E6
:100090000E16061C8E160E18502886180E1452289E
:1000A000861C55287C20CF204B28861C55280E12F4
:1000B0000A303D213A28173090003B309100323011
:1000C00092000C3093001F309400633095000800BC
:1000D000023090000030910001309200083093000F
:1000E0001B3094000630950008000C080D04031D19
:1000F00008008E19031108009E0A10309A00203063
:100100009B000630B6009B20B60B832821162316D1
:100110000E1E8D28A016A216A416A616A816861DB9
:100120009A28A0160C301002031C9A281E199A282F
:100130002112231208001A08840000089C001030C5
:100140001A02031DB228861DB2280C309C08031D1C
:10015000AB289C07B2281C020319B228031CB22842
:100160000C309C029D010A309C02031CB9289D0A98
:10017000B4289C07C0201C089D00C0209A0A0800D3
:100180001B0884001D0880009B0A0D081A02031931
:1001900000178D08031D08008E1900170800203075
:1001A0009B008D080319DB2813300D02031CE62881
:1001B00026309B00E6288E19E6288C080319E628CD
:1001C000120A02390319E62826309B00752003190C
:1001D000EB2850303D210621E9303D2116303D21EC
:1001E0002C301B02031DF62820309B0006217520B1
:1001F000031D0800F3303D210E1A01298E1A032930
:10020000080016303D2116303D210800FF303D2109
:1002100016211B08840025212A303D2125212A3062
:100220003D212521162104089B0008001B0884009D
:100230000630B60000083F39203A031D21291E3040
:100240003D21840AB60B1A2908002A210F303D21CE
:100250002A21080000083F39203A03193B29001FD2
:1002600033291E193529000885000A303D210F3039
:10027000850032303D21840A0800B5000130B40009
:100280008530B300B30B4229B40B4029B50B3E298E
:1002900008000B1D5E290615960003089700040848
:1002A0009800FC308E056921B321D4210B11180868
:1002B000840017088300160806110900B6013608E5
:1002C00085000A303D210F30850032303D21B60ACD
:1002D0005F298E190800B00B08004B30B000B10840
:1002E00003197729B10B7729B00A0030B100920ABF
:1002F0000E188E153C301202031C080092010E18D5
:100300000800910A3C301102031C080091010E18EC
:100310000800900A18301002031C080090010E1803
:100320000800940AA929031C0800013094000E1843
:100330000800930A0D301302031C080001309300DB
:100340000E180800950A64301502031C0800950178
:10035000080003301505031DFF3003190B30130788
:100360000520140293298618CC29B208031DC1293F
:100370008D08031DC1298E1DC1294B30B0008E117F
:100380000E1538303202031DC7298E140E15FF30AA
:100390003202031DB20A0800B20803190800B201B4
:1003A0000E1D0E140E1108008D08031DE0290E1CF1
:1003B000DB298C0908008E1C080010308D00080015
:1003C0000E1CF8299E0110300D02031989291130E5
:1003D0000D020319812912300D02031977291330F8
:1003E0000D020319992914300D0203199129A2292C
:1003F0008E1C080004309E008D0A16300D02031C6E
:0604000008008D019229A5
:0207FE005E2972
:02400E00F23F7F
:00000001FF
